:100000000C9441000C945E000C945E000C945E0015
:100010000C945E000C945E000C94A9000C945E009D
:100020000C945E000C945E000C945E000C945E00D8
:100030000C945E000C945E000C945E000C945E00C8
:100040000C945E000C945E000C945E000C945E00B8
:100050000C945E004C696E6534004C696E6533002B
:100060004C696E6532204142434445464748494AFF
:10007000004C696E6531206162636465666768691A
:100080006A0011241FBECFE5D4E0DEBFCDBF10E073
:10009000A0E6B0E0E2E7F4E002C005900D92A036E1
:1000A000B107D9F710E0A0E6B0E001C01D92A63A72
:1000B000B107E1F70E946E000C9438020C94000026
:1000C0009C01E0EAFFE003C0CF010197F1F7215066
:1000D00030408FEF2F3F3807B9F708950E94C401D1
:1000E0001FBC8EB58C608EBD1DBC1CBC8DE390E02A
:1000F0009BBD8ABD89B7806189BF78940E947101D8
:1001000088EE93E00E94600061E081E00E94660159
:1001100081E790E00E94000261E082E00E946601B7
:1001200080E690E00E94000261E083E00E946601A8
:100130008AE590E00E94000261E084E00E9466018E
:1001400084E590E00E94000280E197E20E94600056
:10015000D5CF1F920F920FB60F9211242F933F937A
:100160004F935F936F937F938F939F93AF93BF93BF
:10017000EF93FF930E942101FF91EF91BF91AF9107
:100180009F918F917F916F915F914F913F912F91AF
:100190000F900FBE0F901F901895F894209160005B
:1001A000E22FFF279091A30034E0EE0FFF1F3A9556
:1001B000E1F7EF59FF4FE90FF11D808378949F5FBE
:1001C0009093A300903150F01092A300822F8F5F84
:1001D00080936000843010F01092600008950E94B7
:1001E000CD000895C29A85E08A95F1F7C2980895E6
:1001F000992780FF02C0AF9A01C0AF9881FF02C06B
:10020000AC9A01C0AC9882FF02C0AE9A01C0AE9811
:1002100083FF02C0AD9A01C0AD980E94F20008951C
:100220001F93182F82958F700E94F800812F8F7076
:100230000E94F8001F910895C0980E941001C09A72
:1002400008958091A500882339F08091A5000E942F
:100250001C011092A5000895E091A200FF27809153
:10026000A40044E0EE0FFF1F4A95E1F7EF59FF4F5E
:10027000E80FF11D80810E9410018091A4008F5F22
:100280008093A4008091A4008031F8F01092A40023
:100290008091A2008F5F8093A2008091A2008430A1
:1002A00010F01092A2008091A200823059F08330A9
:1002B00019F0813019F404C080ED05C080E803C056
:1002C00080EC01C080E98093A500089581508430BE
:1002D00038F46150603120F46093A3008093600093
:1002E0000895F89440E050E016C0FA0164E0EE0F83
:1002F000FF1F6A95E1F7EF59FF4FE20FF31F80E20E
:1003000080832F5F3F4F2031310579F74F5F5F4F7B
:100310004430510519F020E030E0E7CF1092A20000
:100320001092A40080E88093A50078941092600059
:100330001092A30008959C01E0EAFFE003C0CF0102
:100340000197F1F7215030408FEF2F3F3807B9F771
:10035000089582E00E94F80082E00E94F80088E0A0
:100360000E94F80085E090E00E949B0108959C01A6
:1003700095E003C0892F8A95F1F7215030408FEF27
:100380002F3F3807B9F70895B89ABA9AC098C2981B
:100390001092A5001092A2001092A400109260008A
:1003A0001092A300A79AA49AA69AA59A8FEF90E01C
:1003B0000E949B010E94A90188E00E941C0182E327
:1003C00090E00E94B70181E00E941C0185E090E06E
:1003D0000E949B0186E00E941C0182E390E00E9443
:1003E000B7018CE00E941C0182E390E00E94B701FB
:1003F00084E10E941C0182E390E00E94B70108950D
:10040000CF93DF93EC0128C0853B61F1863B38F444
:100410008D3011F1803BB9F08A30B9F41DC0843EB3
:1004200051F0853E18F48F3D81F40BC0863F29F0D2
:100430008C3F59F404C081EE16C08FEE14C085EFD6
:1004400012C082EE10C08FED0EC09927282F88238E
:1004500019F0822F0E94EF00FE01219684918823DB
:1004600099F603C084EE282FF4CFDF91CF91089541
:02047000FFCFBC
:00000001FF
